:2002000018308A00932B0000FFFF2D1D0C1C6629101067308E07F0300318013E8F071014CF
:200220000C102A148316A00A0319A10A0319A20A0319A30A450803196629FF3E031944290B
:20024000FF3E03193129FF3E03193829FF3E03194229CC01CB014808CA0007150430C500A5
:200260006629CA0B66294608CA00071503302F29CA0B66294908FE39031D5D29460846079F
:20028000CA002D29CA0B66294B084C02031D4D29CC01CB01C50107156629CD304B078400C6
:2002A00083130008C900CB0AFE3903192B29FE3C031D5D29C90148086029460849184708DA
:2002C000CA0007110310C90C02302F29831203130408FC008C1E7D29B0304B078400831777
:2002E0001A0880004B08013E3F394A3C03196A294B08013E3F39CB006A297C0884008C120F
:200300000C2809000A148A100A1182077D3468344E343E340A148A100A118207A034A034FF
:20032000C034E0340A148A100A1182074B345234563420344B34523443343234203400340C
:200340000A148A100A118207563431342E3436343B3400340A148A100A1182074B3459347B
:2003600020343C3400340A148A100A118207FE34FD34FB340A148A100A11820700340034D3
:200380000034003400342234003400342D34003468342A34733461340A342934FF343E34F8
:2003A0003C343834303420342134233427342F34003400340034313400344C34003406341C
:2003C000113415340934023414340B34103404341E340D341234073405340F3416341B34F0
:2003E0000A34083403340C3418340E3419341D341334000000000A108A140A11023E03186B
:200400008A0A8200013400340A34003464340034E8340334103427346B08831203178D007E
:2004200083168C130C14831203170C08F80003130034DA0803191F2A0B305A07202A5908D1
:20044000E800680E8800F0308805DA0803192A2A201E2F2A0310680D403EE900332A0310C1
:200460005A0D603EE9006908E90AEA00EB000C227808E8006908EB000C227808E700A01D11
:20048000432A7830442A70305B07E9006908EB000C227808E804670893008316140C031C1E
:2004A0004E2A8312680893008316140C031C552A83128714871000346608EB000C227808D3
:2004C000E800680F852A660803178D000313670803178C0083168C130C15831203130B08B7
:2004E000F7008B138316031755308D00AA308D008C148C18792A0C117708831203138B047E
:200500006608EB000C227808E8006808F8000034E501FF30831685003F30860091308700E0
:200520000F3088000130890081132030840083130408603C031C9F2A8001840A982AA0300B
:20054000840083130408E93C031CA92A8001840AA22A83122011061A2015201007182014E5
:20056000A010851AA014A0110818A015201288182016A012071EA0162017A0178819C22AE2
:200580000130E5070819C62A0230E5076508E600CB01CA01AD010330E605613066078400D7
:2005A000831300088316990026309800903083129800E6018C1AE60A1A08E60083168C16D0
:2005C000831220080739073A0319EA2A013A0319F12AF62A83160108C0390338810083122F
:2005E000F62AFF30831688008312F62AA01DFA2A0330FB2A0730B100871094123030940084
:200600004030831694008312192220080739031D102B83161F149F141F119F11152B831276
:2006200083161F109F141F119F111F1383121F179F1383169F1783121F14E6011930E70082
:200640005C227808C6000130E600E7015C227808AF000230E6004630E7005C220330E6001E
:200660000130E7005C227808DE000430E6000330E7005C222A1178182A15AA100130831646
:20068000C50083122816AB018316A701A601A501FA30A400AB01AA01A901A800AF01AE01B2
:2006A000AD01AC01B301B201B101B001B701B601B501B401BB01BA01B901B801A301A2010A
:2006C000A101A0018530831290000F308F0060308E0083160C14C03083128B045E0882213B
:2006E000F800E50007110C3097000030F8000638920065088316920003108312650DE701A0
:20070000E600E70CE60CE70CE60CE70C66089500E70C670C3039F7001708CF397704970034
:2007200083160715043083128900A1108A150A16AA2B86196B2C0F30E60066308400831362
:2007400000080319B12B0130F800F701F70BA62BF80BA52B4A30F700F70BAC2BAF2B800B23
:20076000A32B86196B2C06308900E50165083F3C031CE32B40306507E60065080A168A15CD
:2007800068250A128A11E700660803178D000313670803178C0083168C130C1583120313EA
:2007A0000B08F7008B138316031755308D00AA308D008C148C18DA2B0C11770883120313D5
:2007C0008B04E50AB62B8901E50165081F3C031C392CA0306507E60065080A168A15AC25DF
:2007E0000A128A11E700660803178D000313670803178C0083168C130C15831203130B0804
:20080000F7008B138316031755308D00AA308D008C148C18092C0C117708831203138B04C8
:20082000C0306507E60065080A168A15AC250A128A11E700660803178D0003136708031727
:200840008C0083168C130C15831203130B08F7008B138316031755308D00AA308D008C1494
:200860008C18302C0C117708831203138B04E50AE52B06308900E50165083F3C031C692C62
:20088000C0306507E60065080A168A15C0250A128A11E700660803178D00031367080317B3
:2008A0008C0083168C130C15831203130B08F7008B138316031755308D00AA308D008C1434
:2008C0008C18602C0C117708831203138B04E50A3C2C043089008A150A16AF2BEF01F00184
:2008E0006E08EE03003A0319A62C6D08ED0A363E8400831730300002F1007108093C03183F
:20090000862C6F08F8007008F900AA2C03106F0DF200700DF3006F0DF900700DFA00F90D8C
:20092000FA0DF90DFA0DF830F90579087207F4007308F5007A0803187A0FF5077108740709
:20094000EF007508F0000318F00A702C6F08F8007008F9000034013003179300383092009E
:200960000313B801380803171007840083131118831700080313ED00380803171207840058
:20098000831313188317000803136D02031DD12C38080A3C031DCF2C0030F800D32CB80AC8
:2009A000B22C0130F8000034013003179300383092000313B80138080A3C031CFD2C380847
:2009C00003171007F8001108FA000318FA0A78080313ED0038080317120784008313131881
:2009E000831700080313EF006D08840083137A1883176F088000B80ADB2C0B300317100769
:200A000084008313111883178001031300341030F100F701FA01EE0CED0C031C152D6F083F
:200A2000F7070318FA0A7008FA07FA0CF70CF90CF80CF10B0B2D00348B13831203138A01D2
:200A4000FC20831203138A01FD2003179908031D4C2D160803194C2D9708031D212D831779
:200A60001A30840018088D0000088C0083168C130C1555308D00AA308D008C140C118C1834
:200A80003F2D83128D0A840A960B342D03130C1E472D47309900212D8313031383128B1739
:200AA0008A150A12B72AF701F8016D0803106E18F707F70CF80CEE18F707F70CF80C6E1904
:200AC000F707F70CF80CEE19F707F70CF80C6E1AF707F70CF80CEE1AF707F70CF80C6E1BE2
:200AE000F707F70CF80CEE1BF707F70CF80C00348316981C8A2D83124D084C020319892DA1
:200B000090304D078400831700089900CD0A1F30CD05831683122D080319A72D103A031951
:200B2000AE2D013A0319AE2D033A0319AE2D323A0319D72D013A0319D72D033A0319D72D30
:200B4000013A0319D72D073A0319D72DDE2D0317B6010313C9011030AD00E02D4A084B0284
:200B60000319D62D4A08CA0AB03E840083170008E5003F30CA054908C90A363E8400831743
:200B800065087F3980003630490784008317800165083B3C031DCF2D1030AD07E02D490809
:200BA000373C0318D52DAD01E02DAE2DE02DAE018A1500288A117808AD00E02DAD01E02DFC
:200BC0008A150A16B42B0B138B138B1BE42D703081000B11211009188B2E3A260B198B2E7F
:200BE000091CEE2D3A263A263A266C26B4006C26B500B6003408213C03190B2E3408203CCC
:200C000003190F2E3408343C0319152E3408353C0319252E382E3508B3002216382E350823
:200C20000F39013EB200A215382E5B0DF700F70DFC30F70577085B0735070A168A150025D2
:200C40000A128A11F800B6002D2E35085F073105DF00B600A2162D2E21143608831609102E
:200C600083127B2609143A268316091483128B2E6C268B2E4930B8004526B8024526B802F7
:200C80005326B802B80B422E00348C1E01348317B0304B0784001A088000CB0A3F30CB05D5
:200CA0008313000005340C1C0134101067308E07F0300318013E8F0710140C10831683163A
:200CC000A00A0319A40A0319A80A0319AC0A831283122A1400000834B5018030B700350802
:200CE00009183704B5003A263A260310B70C031C6F2E350808008030B7003608370503194F
:200D0000832E0914842E09103A263A260310B70C031C7D2E0034C0308B048A150A12D82B69
:200D2000690DF700F70DF70DF830F7051F08C73977049F001030F700F70B9C2E00001F15A2
:200D40001F19A02E1E08FA0083161E08F8007A08F900831200348316A408031DB82EA5087A
:200D6000031DB82EA608031DB82EA7080319DF2E27082302031CDF2E031DCE2E26082202F3
:200D8000031CDF2E031DCE2E25082102031CDF2E031DCE2E200824020318DF2E2808A40722
:200DA00029080318290FA5072A0803182A0FA6072B0803182B0FA707831222158316AC0881
:200DC000031DEB2EAD08031DEB2EAE08031DEB2EAF080319122F2F082302031C122F031D0D
:200DE000012F2E082202031C122F031D012F2D082102031C122F031D012F20082C02031840
:200E0000122F3008AC0731080318310FAD0732080318320FAE0733080318330FAF07831230
:200E2000A3158316B408031D1E2FB508031D1E2FB608031D1E2FB7080319452F3708230230
:200E4000031C452F031D342F36082202031C452F031D342F35082102031C452F031D342F8E
:200E6000200834020318452F3808B40739080318390FB5073A0803183A0FB6073B08031869
:200E80003B0FB70783122316831683128A150A16BC2B01304C071F394D020319582F90301A
:200EA0004C078400831773088000CC0A1F30CC050034AA185F2F7208F30049277E2FAA1CFC
:200EC0007E2F83164C081E3C031C7D2F2030F20272083A3C031C7D2F4C08CC0ACD3E84009B
:200EE000831372088312BA21F80080008316C508031D7D2FCB010130C500831200346A08CB
:200F0000EA03003A03198F2F6908E90A0A168A1552240A128A11EC00F20059277F2F003440
:200F2000EC080319C22FEC0303106C0DF100710AF921FA007108F921EF007A08F000EE01D2
:200F400070086B02031CB22F031DAA2F6F086A02031CB22F6F08EA027008031C700FEB026A
:200F6000EE0AA02FEE08031DBB2FED080319BB2FEC08031DC12F30306E07F100F200592773
:200F8000ED01902F0034580DE600E60DFC30E605D8016608F800003447083F393F3C03194A
:200FA000D52FE7018A1500268A11480FD82FDF2F4808C7000130E7008A1500268A118A154B
:200FC0000A16152B4708F039031DEE2F0730C7050230E7008A1500268A11F82F4708FF3AD1
:200FE0000739013EC7000330E7008A1500268A118A150A161B2BFFFFFFFFFFFFFFFFFFFF36
:2010000003173608603C03180C2836087A3C031C0C283608DF390D2836080313E600031767
:201020003708603C03181B2837087A3C031C1B283708DF391C2837080313E7004130660270
:20104000E83E03189B2B183E9E2B67084E3C031D3928031738080339FF3E0313E8000030EF
:20106000271A013068020319392827126818271624170030F8009B2B6708473C031D492875
:201080000230ED00EE008A116E248A157808BA0024150030F8009B2B6708533C031D702860
:2010A000E8016808093C031C6C282C306807ED000130EE000318EE0A02306807363E84005C
:2010C00083170008F0006D08840083136E18831770088000E80A5128A3160030F8009B2BC5
:2010E0000030F8009B2B6708413A03198428033A03199D28103A0319B628063A0319C828A2
:20110000033A0319DA280A29013003179100143090008A110313AB248A15F80803199A2894
:20112000013003179100143090008A110313D4248A1522170030F8009B2B013003179100B4
:20114000203090008A110313AB248A15F8080319B328013003179100203090008A1103132C
:20116000D4248A15A2170030F8009B2B0317380801390313E8000030A618013068020319FA
:20118000C528A6106818A61423140030F8009B2B0317380801390313E8000030261901301B
:2011A00068020319D728261168182615A3140030F8009B2B0230ED000430EE008A116E24A5
:2011C0008A157908EA007808E90069084102031DED286A0842020319F2286A08C200690822
:2011E000C100251603173C080F390313E80068083D020319FE286808BD00A51603173D0817
:201200000F390313E80068083E0203190A296808BE0025170030F8009B2B6708543C031D12
:2012200030290230ED000330EE008A116E248A157808E80068083B02031921296808BB00A3
:20124000251403173B0801390313E8000030261A0130680203193029261268182616251413
:201260000030F8009B2B6708463C031D292A2D08203C031D6C29031748080313E80013302B
:20128000ED000430EE008A116E248A157908EC007808EB0068082D3C031D5C296C08EE00BB
:2012A0006B08ED00FF30F000EF008A1107258A157908EC007808EB006B084302031D64291D
:2012C0006C084402031969296C08C4006B08C300A4142330F8009B2B2D08233C031DEB29A7
:2012E0000317540801390313E8000030A6180130680203197F29A6106818A61423140317B2
:20130000560801390313E800003027190130680203198E29271168182715A417271D9429A9
:201320000030A61C013097290030A6180130E80000302619013068020319A229261168181B
:201340002615A3143030031752020313E800E8080319AC292619B129E808031DC829A61C12
:20136000C829013003179100203090008A110313AB248A15F8080319C729013003179100B9
:20138000203090008A110313D4248A15A217E829E8080319CD29261DD229E808031DE829FA
:2013A000A618E829013003179100143090008A110313AB248A15F8080319E8290130031717
:2013C0009100143090008A110313D4248A1522172430F8009B2B2D08243C031D292A0317F3
:2013E00053080F390313E800A11668083C020319FC2922146808BC0003175508013903137D
:20140000E8000030A61B0130680203190B2AA6136818A617A51703174D0801390313E800AE
:20142000003027180130680203191A2A271068182714A31703174E0801390313E8000030BE
:20144000A718013068020319292AA7106818A71424140030F8009B2B6708533A0319372A32
:201460000A3A03194B2A0B3A0319592AB72A0230ED000330EE008A116E248A157808E8005E
:201480002117680845020319482AA2146808C5000030F8009B2BA81D562A03173808323CE9
:2014A0000319542A0313562A031321160030F8009B2B2D08203C031D6C2A03173808303CB4
:2014C000031D6D2A3908303C031D6D2AB6010313C9011130F8009B2B031703132D08213C99
:2014E000031D812A03173808373C031D822A3908333C031D822AB6010313C9011230F8003B
:201500009B2B031703132D08223C031DB72A03173808603C0318932A38087A3C031C932AA1
:201520003808DF39942A38080313E8006808553A0319A42A103A0319A72A133A0319AA2AFA
:20154000153A0319AC2AB72A8A01FF28B72A8A111C2D8A15A115B72A1D3003179100900133
:201560002030930092018A010313FE28B72A0030F8009B2B67084B3C031DCD2A03173808F8
:2015800001390313E8000030A619013068020319CD2AA6116818A61523170030F8009B2B5C
:2015A0006708443C031DE12A031738080F390313E800A11668083C020319E12A6808BC00B9
:2015C00022140030F8009B2B6708423C031D032B0317380803390313E80068083F0203194B
:2015E000F42A6808BF0024160317390801390313E80000302618013068020319032B261048
:2016000068182614A4160030F8009B2B6708413A03190E2B023A0319202B3F2B03173808C2
:2016200001390313E8000030A61A0130680203191D2BA6126818A61625150030F8009B2B67
:201640000230ED000330EE008A116E248A157808E80003173B1C372B03136808ED000A3096
:20166000EE008A1153258A157808E800031703136808400203193F2B6808C0002315003062
:20168000F8009B2B6708413A03194A2B153A03195C2B6B2B0317390801390313E8000030C6
:2016A000261B013068020319592B261368182617A5150030F8009B2B031738080139031366
:2016C000E800003027180130680203196B2B271068182714A3170030F8009B2B6708513CD0
:2016E000031D822B0230ED000330EE008A116E248A157808E800680839020319822B6808C5
:20170000B900A4150030F8009B2B6708543C031D982B0317380801390313E8000030A71806
:20172000013068020319982BA7106818A71424140030F8009B2B8A110A12DA2D0A148A149D
:201740000A11820725283C289B2B4C289B2B73280D299B2B33299B2B2C2ABA2AD02AE42A39
:201760009B2B062B9B2B422B6E2B9B2B9B2B9B2B9B2B852B3208E80020080739E7006708FE
:20178000073A0319D62B013A0319DA2B033A0319E82B053A03199E2C013A0319A02C033A9E
:2017A0000319A02C013A0319A02C292D8A11E32D8A15292D080EF7000F30F70577080F3919
:2017C000E800350868020319292D6808B500FA2CA618FC2B221FFC2B031717080F390313D9
:2017E000E700670EE900F030E905031718080F3903136904E700112CA61C102CA21F102C72
:20180000031723080F390313E700670EE900F030E905031724080F3903136904E700112C9D
:20182000292D6708013A0319582C033A03195B2C013A03195E2C073A0319612C013A031906
:20184000642C033A0319672C013A03196A2C0E3A03196D2C193A0319702C033A0319732C1F
:20186000073A0319762C0C3A0319792C383A03197C2C013A03197F2C053A0319822C013AE6
:201880000319852C023A0319882C0F3A03198B2C013A03198E2C793A0319912C013A03195F
:2018A000942C033A0319972C013A03199A2C9D2C0130E8009D2C0130E8009D2C0230E80088
:2018C0009D2C0A30E8009D2C0A30E8009D2C0330E8009D2C0330E8009D2C0430E8009D2CBC
:2018E0000430E8009D2C0530E8009D2C0530E8009D2C0630E8009D2C0730E8009D2C073031
:20190000E8009D2C0830E8009D2C0830E8009D2C0930E8009D2C0930E8009D2C0930E8004F
:201920009D2C0B30E8009D2C0B30E8009D2C0B30E8009D2C0B30E8009D2CFA2C0130E700F0
:201940000330E7056708E9008A1190268A157908E6007808E5006708E9008A1190268A150C
:201960007808E50779080318790FE6076708E9008A1190268A157808E50779080318790F12
:20198000E6076708E9008A1190268A157808E50779080318790FE607E60CE50CE60CE50CCF
:2019A000E60CE50CE60CE50C0F30E60567088A118A218A15F800E7006708E70AE900EB00D0
:2019C0008A110C228A15E608031DEA2C650878020318EC2CE70ADC2C6708EB008A110C2245
:2019E0008A157808E800350868020319292D6808B500FA2C68080B3C03181E2D68080C3CA7
:201A0000031D042D0130E80068080D3C031D0A2D0230E80068080E3C031D102D0330E80000
:201A200033080739680203191D2D68080739F700F83033057704B3002216292DF830330538
:201A4000B3002216320868020319292D6808B200A2158A150A16B82B2A1CDD2D2A10E5019A
:201A60006508033C031CDD2D0310650D503EE700E8010318E80A6508FC3E0318512D043E1F
:201A8000E02DE6018618E60A512DE6010618E60A512DE6010619E60A512DE6018619E60AE9
:201AA000512D670884008313681883170008FC3E0318DB2D043EF82DE608031D6C2D670823
:201AC000840083136818831701308000670784008313681883178001DB2D013067078400D3
:201AE000831368188317800A0008093C0318842D67088400831368188317E6080319822D37
:201B00000030832D02308000DB2D8316C5080319952D83126708840083136818831703307C
:201B2000800005308316C500CF2D0130831267078400831368188317800A00087C3C031CC5
:201B4000B92DE6080319B82D6708840083136818831780016508FC3E0318B82D043EE82D8E
:201B60002914B82D2915B82D2916B82D2917B82DCE2D670884008313681883170330800086
:201B80006508FC3E0318CE2D043EF02DA914CE2DA915CE2DA916CE2DA917CE2D8316831215
:201BA000DB2DE6080319DA2D670884008313681883178001DB2DE50A302D8A150A16C02BEA
:201BC0000A148A100A158207412D452D492D4D2D0A148A100A158207B02DB22DB42DB62DF5
:201BE0000A148A100A158207C62DC82DCA2DCC2D0A148A100A1582075C2D6D2D852DD12D7A
:201C00006708ED000330EE008A1153258A15023078070A1600240A12F800E8006708ED0048
:201C20000330EE008A1153258A1578080A1600240A12EA00F3008A1149278A156708ED000E
:201C40000330EE008A1153258A15013078070A1600240A12EA00F3008A1149278A156808AA
:201C6000F83E0318902E083E962E0130C70530304707E900F3008A1149278A15902E3030FC
:201C80004707E900F3008A1149278A1530304807E900F3008A1149278A15902EEB01470842
:201CA000EA000330EC00ED018A1190278A15902EEB014708EA000230EC00ED018A119027FB
:201CC0008A15902E2030F3008A1149278A156808073C031D702E3C30F3008A1149278A1540
:201CE000283048070A1600250A12F800F8080319852E4808C80A283E0A1600250A12EA0042
:201D0000F3008A1149278A15702E6808073C031D8E2E3E30F3008A1149278A15902E902E72
:201D20003B30F3008A1149278A1500340A108A140A1582078F2E352E372E3F2E582E4E2E13
:201D4000622E622EDD080319A82E5D08F800CE2FA2080319DB2E221CB12E22102B30F800C1
:201D6000CE2FA21CB72EA2102930F800CE2F221DBD2E22113730F800CE2FA21DC32EA211A7
:201D80000330F800CE2F221EC92E22120230F800CE2FA21ECF2EA2120430F800CE2F221FAE
:201DA000D52E22132030F800CE2FA21FDB2EA2132130F800CE2FA90803191E2F291CE82E6C
:201DC00029108A11C3278A1509307807F800CE2FA91CEE2EA9100530F800CE2F291DF82EC9
:201DE00029118A11C3278A150A307807F800CE2FA91DFE2EA9110630F800CE2F291E082F82
:201E000029128A11C3278A150B307807F800CE2FA91E0E2FA9120730F800CE2F291F182F3A
:201E200029138A11C3278A150C307807F800CE2FA91F1E2FA9130830F800CE2FA3080319CD
:201E4000512F231C272F23102230F800CE2FA31C2D2FA3102330F800CE2F231D332F231107
:201E60002F30F800CE2FA31D392FA3113830F800CE2F231E3F2F23123930F800CE2FA31ED2
:201E8000452FA3121F30F800CE2F231F4B2F23132A30F800CE2FA31F512FA3133130F80043
:201EA000CE2FA4080319842F241C5A2F24103330F800CE2FA41C602FA4103430F800CE2FF9
:201EC000A41D662FA4113230F800CE2F241E6C2F24122C30F800CE2FA41E722FA4122D30C6
:201EE000F800CE2F241F782F24131D30F800CE2FA41F7E2FA4133530F800CE2F241D842F15
:201F000024111E30F800CE2FA5080319B72F251C8D2F25102730F800CE2FA51C932FA510E4
:201F20003B30F800CE2F251D992F25112E30F800CE2FA51D9F2FA5113030F800CE2F251ED0
:201F4000A52F25122430F800CE2FA51EAB2FA5122530F800CE2F251FB12F25132630F800E5
:201F6000CE2FA51FB72FA5133630F800CE2FE0080319CC2F601CC02F60103D30F800CE2F6B
:201F8000E01CC62FE0103E30F800CE2F601DCC2F60113C30F800CE2F0030F8008A150A16CC
:201FA0005D2A0430E70000268A150A16202B0530E70000268A150A16242B1530E90006309B
:201FC000EA008A117F278A1530304707E600F2008A1159278A153B30F2008A1159278A15E0
:201FE0008A150A16282B1730E70000268A150A16382BFFFFFFFFFFFFFFFFFFFFFFFFFFFF67
:202000008316C50803190628013007280030F8008312281378182817A8193828A11E3328AE
:202020003C08CE002A1933283C08013A03192828033A03192828013A03192B28043A031958
:202040002B28013A03192E280F3A03192E2831288030AF0033284030AF003328C030AF0099
:202060003328AF013328211F38284508CF00A117221E4628F701A719F717330877068039A1
:2020800003194628A711B31BA715A514A8080319F228A81C5A282210A11E5128A810A112BA
:2020A0005A28221D5A28B00A3008043C03185A28BC01A810281D6128A210211F6128281117
:2020C0002113281EAD28A21D67283208D900221E6C2833080739DA00221DAA2822112119A9
:2020E00087282115A01E7F28E9011230EA000A127F270A16A81428150130DC0086282812B0
:20210000A8102811A1170130AB00AC01AA28A81890282819902828120130AB00AC01AA28B5
:202120005C08093C031C9E28A01E9E28E9011230EA000A127F270A16DC0AAA280A30AE00F5
:202140002812A8102811BC08031D2115C5010130AB00AC01A11221136A29A81DE52822106D
:20216000A210211ECE2821124F08C700A21021131030E7000A128A1500260A168A11281541
:202180004E08C7000530E7000A128A1500260A168A11A814A1122210A811E428221DE428B9
:2021A000AE0A2E080A3C0318DB280A30AE002111BC01C501E42822111230E9000330EA00A9
:2021C0000A127F270A16A8156A29A81EF228831603178C1CEE2883120313F228831203130C
:2021E0000D12A812A11D1129E50165080A1292210A16003803190229E50AF2000A125927D0
:202200000A16F528E50165080A12A0210A16003803191029E50AF2000A1259270A160329DB
:20222000A111221D6829221121192429201F2429AE0A0230EB000A120C220A162E087802E7
:20224000031824292816AE01D808031D34295908320203192D29A11C312904308900A11040
:20226000342906308900A1143C084E0203194D29CE08031D3E293C08CE004D29BC080319A2
:202280004D29A01E4D294E08C7002930E9000330EA000A127F270A16A81445084F020319C0
:2022A0006829CF0803195629A11B59294508CF006829C50803196829A01E68294F08C70049
:2022C0001030E7000A128A1500260A168A112815A11221138A150A16C32B1B30E900043002
:2022E000EA000A127F270A16C70803198B290130C800261A81293230F2000A1259270A1680
:202300008A293430F2000A1259270A163B08043C0319C8019729C80803199129303048077B
:2023200092293230E600F2000A1259270A16C80803199C2931309D293030E600F2000A12C0
:2023400059270A163B30F2000A1259270A168A150A162C2B47083F393F3C031DB1293F082B
:20236000C7000330C705480FB829C8012618C80A0130C8050830E7000A128A1500260A1668
:202380008A118A150A16302B47083F393F3C0319D0290930E7000A128A1500260A168A1175
:2023A000480FD329DC294808C7000A30E7000A128A1500260A168A118A150A16342B470884
:2023C0003F393F3C0319EB290B30E7000A128A1500260A168A11480FEE29F5290C30E7006D
:2023E0000A128A1500260A168A118A150A163C2B47083F393F3C031D052A0D30E7000A124A
:202400008A1500260A168A11162A470B0F2A0E30E7000A128A1500260A168A11162A0F3031
:20242000E7000A128A1500260A168A118A150A16402BA11F282AC708031D212A4508480707
:20244000C7001030E7000A128A1500260A168A118A150A16442BC7080319312A4708C60069
:20246000332A4808C6074608093C031C392A0A30C6004608323C03183F2A3230C60003174B
:202480008D010313460803178C0083168C130C15831203130B08F7008B13831603175530C0
:2024A0008D00AA308D008C148C18542A0C117708831203138B04A8168A150A16482BC708D1
:2024C000031D652A40084807C7001130F2000A1259270A168A150A164C2B1230E7000A1285
:2024E0008A1500260A168A118A150A16502B470B812A1330E7000A128A1500260A168A115F
:202500008D2A47083F393F3C031D8D2A1430E7000A128A1500260A168A118A150A16542BE6
:20252000A11F992A1530E7000A128A1500260A168A118A150A16582B6D08ED03003A031953
:20254000B22A6C08FA006B08EB0A0319EC0A840083137A1883170008EE00F2000A125927ED
:202560000A169C2A0034E9080319B82A4E30B92A4630EA00F2000A1259270A16003469083E
:20258000F80168020318C72A6808F700D32AF7010830EA00E80DF70D690877020318F70059
:2025A000F80DEA0BCA2A00344708DB3E0318632D253E712D2830C8074808C80A8A150025D8
:2025C0008A11F800E700E7080319EC2A6708F2000A1259270A16DC2A632D4808F2000A124F
:2025E00059270A16632D2F0EF700F70CF70C0330F7057708313EE900F2000A1259270A16BD
:20260000632DA618322B0230E70014306707840083170008303C031D162BE70A14306707AE
:20262000840083170008303C0319E70A14306707E8000130E9000318E90A6708053CEA009F
:202640006908EC006808EB006A08ED009C22632DA618572B0130EC001930EB000330ED0064
:202660009C22632D0230E70020306707840083170008303C031D452BE70A203067078400E0
:2026800083170008303C0319E70A20306707E8000130E9000318E90A6708053CEA00690846
:2026A000EC006808EB006A08ED009C22632D0130EC002530EB000330ED009C22632DA61C99
:2026C000632B4230642B4130E800F2000A1259270A16632D261D6E2B42306F2B4130E80093
:2026E000F2000A1259270A16632D003027190130E800E900B322632DBD080319822B3030D7
:202700003D07832B4630E800F2000A1259270A16632DBE0803198F2B30303E07902B4630B9
:20272000E800F2000A1259270A16632D261E9B2B30303B079C2B4630E800F2000A12592714
:202740000A16632DEB014508EA000230EC000130ED000A1290270A16632D0030A6190130C7
:20276000E800E900B322632D01303C02F73E0318002C093E642DC8080319C02B0130C12B6C
:202780000330E8002C30E9006808EA000A127F270A16002CC8080319CF2B0130D02B03302C
:2027A000E8002F30E9006808EA000A127F270A16002CC8080319DE2B0130DF2B0230E80037
:2027C0003230E9006808EA000A127F270A16002C3630E9000230EA000A127F270A16002CCD
:2027E0003430E9000230EA000A127F270A16002C3530E9000230EA000A127F270A16002CEA
:20280000632DBF080319072C30303F07082C4630E800F2000A1259270A16632D003026182E
:202820000130303EE900F2000A1259270A16632D0030261B0130E800E900B322632D0030CA
:20284000A61A0130E800E900B322632D4008E8000A30E900BF227808E800EB017808EA005F
:202860000330EC000130ED000A1290270A162E30F2000A1259270A164008E8000A30E900C9
:20288000BF2230307707E900F2000A1259270A16632D003027180130E800E900B322632D7C
:2028A0000030A7180130E800E900B322632D0030A61B0130303EE900F2000A1259270A169B
:2028C000632D0030271A0130313EE900F2000A1259270A16632DEB013908EA000330EC00FA
:2028E0000130ED000A1290270A16632D3A080A3C03187D2C0C303A027E2C3A08E700EB01B4
:202900006708EA000230EC000130ED000A1290270A16632D4208EB004108EA000430EC0017
:202920000130ED000A1290270A16632D48080319A02C013A0319A52C033A0319A82CAB2C92
:20294000A718A32C2718AC2CAB2C2718AC2CAB2CA718AC2CAB2C632DC41BBA2C4408EB0013
:202960004308EA000430EC000130ED000A1290270A16D12C4D30F2000A1259270A1643097D
:20298000E8004409E900E80A0319E90A6908EB006808EA000430EC000130ED000A12902751
:2029A0000A16632DE9016908073C031C382D2C306907840083170008E800E81FE42C5230D2
:2029C000F2000A1259270A16E81368083C3C031DEC2C4C30E800312D68083E3C031DF32C43
:2029E0002D30E800312D6808403C031DFA2C2030E800312D68084B3C031D012D4830E800C7
:202A0000312D68084D3C031D082D4E30E800312D6808513C031D0F2D4F30E800312D6808B8
:202A2000563C031D162D5530E800312D6808573C031D1D2D4930E800312D68085A3C031D84
:202A4000242D4330E800312D6808583C031D2B2D4330E800312D68085B3C031D312D523030
:202A6000E8006808F2000A1259270A16E90AD32C632D0030A7190130E800E900B322632D77
:202A80005908E70067080A3C0319E7016708093C03184C2D0730E70730306707E800F20020
:202AA0000A1259270A16632DE80168080A12A0210A1600380319622DE80AF2000A12592711
:202AC0000A16552D632D00340A148A100A158207BB2BCA2BD92B002C002CE82BF02B002C9F
:202AE000F82B0A148A100A158207DA2AED2A632D012B282B032B2A2B322B572B5F2B6A2BA8
:202B0000752B7C2B8A2C962BA22BAD2BB42B012C0E2C182C1F2C262C492C502CAC2C962CA0
:202B20006B2C762CD22C572C612C392D892BF32A402D542DAA103B30F2000A1259270A1656
:202B4000A01EDE2DA11FDE2D3C08CE004508CF003C08033C0319B72D3C08073C0319B72DA9
:202B60001F30E9000430EA000A127F270A164708E6004608C7001030E7000A128A150026CB
:202B80000A168A116608C700E70167080A12AA210A1600380319D22DE70AF2000A12592715
:202BA0000A16C52DD4223E30F2000A1259270A163B30F2000A1259270A16A8158A150A165C
:202BC0005C2BC7080319EE2D4808C7001630E7000A128A1500260A168A11012E4808C80A37
:202BE000283E8A1500258A11F800C700C7080319012E1630E7000A128A1500260A168A116E
:202C0000EE2D8A150A16602B05302B02FC3E03182E2E043E3B2E580B0E2E102E0130112E44
:202C20000030D8002E2E5808023C0319192E02301A2E0030D8002E2E5808033C0319222E46
:202C40000330232E0030D8002E2E5808043C03192B2E04302C2E0030D8002E2ED808031989
:202C6000352E06308900A114382E04308900A1108A150A16642B0A108A140A1582070B2EC2
:202C8000132E1C2E252E4708E7004808E6004708EE004808ED00F001FA30EF000A1207251E
:202CA0000A168316B301B2017908B1007808B0008312470848040319632E0130F700F80194
:202CC000F901FA01672EF701F801F901FA017A088316AF007908AE007808AD007708AC0033
:202CE00083128A150A16682B4708E7004808E6004708EE004808ED00F001FA30EF000A12E1
:202D000007250A168316BB01BA017908B9007808B8008312470848040319942E0130F700AF
:202D2000F801F901FA01982EF701F801F901FA017A088316B7007908B6007808B50077083C
:202D4000B40083128A150A166C2B47080F3A0319B32E0F3A0319B62E013A0319B92E033A7B
:202D60000319BC2EBF2E3208D900BF2E4808D900BF2E4808D907BF2E4808D902BF2ED90834
:202D80000319C42ED91FC62E0B30D90059080B3C0318CC2E0130D9000A1219220A168A1548
:202DA0000A16702BC7080319D82E33080739D92E4808DA000A1219220A168A150A16742BE6
:202DC000E60147080F3C031DE82E5F08DB00212F0330C805C80803191F2F4708073C031CBF
:202DE000F42E2608E600012F47080F3C031CFB2E2708E600012F4708173C031C012FFF3026
:202E0000E6000730C7054708F80003190B2F0310E60CF80B072F0130E605C8034808F800BF
:202E20000319162F0310E60DF80B122F48080A12B3210A16F800DB056608DB04212F4708C3
:202E4000DB000A1219220A168A150A16782B6808DE0068080A1282210A16F800E900003010
:202E6000F8000638920069088316920003108312690DEB01EA00EB0CEA0CEB0CEA0CEB0C29
:202E80006A089500EB0C6B0C3039F7001708CF3977049700033003178D0003135E080317B4
:202EA0008C0083168C130C15831203130B08F7008B138316031755308D00AA308D008C140E
:202EC0008C18602F0C117708831203138B0400344708FB3E03189D2F053EA02FB00129302A
:202EE000E9000330EA000A127F270A16A8149D2F0317AC0126300313E9000330EA000A120D
:202F00007F270A169D2FFF30BA002330E9000330EA000A127F270A169D2F0830E9000430DA
:202F2000EA000A127F270A169D2F3830E9000430EA000A127F270A169D2F8A150A167E2B74
:202F40000A148A140A1582076E2F782F832F8D2F952F4808003A0319B52F023A0319B62FD0
:202F6000013A0319BE2FC92FC62FC62F83163C1CBC2F8312C92F83168312C62F83163C18B2
:202F8000C42F8312C92F83168312C62F47083F39DD008A150A16862B4608E6006608093C93
:202FA000031CD42F0A30E60066082F3C0318DA2F2F30E6000A3066028A1592248A11F80003
:202FC0008316C600460846074607C700460847074607C8008312AA14D4222030F2000A128B
:202FE00059270A16AA108A150A168A2BFFFFFFFFFFFFFFFFFFFFFFFFFFFFFFFFFFFFFFFF17
:2030000001304702EF3E0318D628113ED9282008F839E600480807396604A000D628480879
:203020000139F800A0117818A015D62848080139F800201278182016D62848080139F80070
:20304000A0127818A016D62848080139F800201378182017D62848080139F800A01378183B
:20306000A017D62848080139F800AA117818AA15D62801305E020339E700E8008A1127278C
:203080008A15D62801305E070339E700E8008A1127278A15D628AF01013003178D000313CE
:2030A0002F0803178C0083168C130C15831203130B08F7008B138316031755308D00AA30E8
:2030C0008D008C148C1862280C117708831203138B042A1100302A190130E60004300317AC
:2030E0008D000313660803178C0083168C130C15831203130B08F7008B1383160317553035
:203100008D00AA308D008C148C1884280C117708831203138B04D628480EF700F70DF70DA2
:20312000C030F70577082F07C039AF00013003178D0003132F0803178C0083168C130C1522
:20314000831203130B08F7008B138316031755308D00AA308D008C148C18AC280C1177083C
:20316000831203138B042A1500302A190130E600043003178D000313660803178C008316AE
:203180008C130C15831203130B08F7008B138316031755308D00AA308D008C148C18CE28B6
:2031A0000C117708831203138B04D6288A150A167B2B0A108A100A11820707280F281628DA
:2031C0001D2824282B28D6283228D62839284228D628D628D628D6284B288C28470807393C
:2031E000BD3EE600E7010318E70A470CF700F70CF70C1F30F70577080739F83E03184D29D9
:20320000083E632966088400831367188317480880004D2966088400831367188317480804
:20322000000780004D29660884008313671883174808000280004D296708FA00660884004D
:2032400083136718831748080002031D292901302A290030F80083163C1078183C145F2902
:2032600083124D29660884008313671883170008480480004D2966088400831367188317B7
:203280000008480580004D29660884008313671883170008480680004D296708FA0066081F
:2032A00084008313671883178008031D592901305A290030F80083163C1078183C1483127B
:2032C0008A150A16812B0A148A100A11820702290A2913291C29312932293B294429470873
:2032E0000739BD3EE600E7010318E70A0730C805470CF700F70CF70C1F30F705770807395B
:20330000F83E0318332A083E492ABD304807840083130008EA00660884008313671883175D
:203320006A088000332A660884008313671883170008EA00BD3048078400831300086A07DC
:20334000EB00660884008313671883176B088000332A660884008313671883170008EA00FE
:20336000BD3048078400831300086A02EB00660884008313671883176B088000332A670838
:20338000FA00660884008313671883170008E800BD3048078400831300086802031DD229BF
:2033A0000130D3290030F80083163C1078183C14452A8312BD304807F800FA010318FA0AA1
:2033C0007A08E900660884008313671883170008EA00780884008313691883176A08800048
:2033E000332A660884008313671883170008EA00BD3048078400831300086A04EB006608B8
:2034000084008313671883176B088000332A660884008313671883170008EA00BD3048075A
:203420008400831300086A05EB00660884008313671883176B088000332A66088400831397
:20344000671883170008EA00BD3048078400831300086A06EB006608840083136718831707
:203460006B088000332A6708FA00660884008313671883178008031D3F2A0130402A003016
:20348000F80083163C1078183C1483128A150A16832B0A108A140A11820785299329A929D5
:2034A000BF29DA29F129072A1D2AA808031D902BAB08031D622A0A12A22E0A167808AB006E
:2034C000AC01DD01AB0803198E2B2C08FA3C031C8E2BE60103102C0DAC0A031703178D00ED
:2034E0001E300318013E8F00831683168C170C1400000000831283120C0803130319A62A60
:2035000003132B020319872A2F07031DA92A031703170E0803130313E600031703178D0A4B
:2035200003198F0A831683168C170C1400000000831283120E0803130313C700031703177A
:203540000C0803130313C800A92A0317FF300313E6006608F8007808E5006508FF3A0319BE
:203560000F2BFE3A0319122B033A0319182B013A03191E2B073A0319222B013A0319262BF2
:20358000033A03192A2B013A03192E2B0F3A0319322B013A0319362B033A03193A2B013A5A
:2035A00003193E2B073A0319422B013A0319462B033A03194A2B013A03194E2B1F3A0319E1
:2035C000522B013A0319562B033A03195A2B013A03195E2B073A0319622B013A0319662B06
:2035E000033A03196A2B013A03196E2B0F3A0319722B013A0319762B033A03197A2B013ABA
:2036000003197C2B073A0319802B013A0319822B033A0319842B013A0319882B8C2BFB30E7
:20362000AC008D2B0A128A11CC2F0A168A15902B0A128A11E22F0A168A15902B0A12D12F9C
:203640000A16902B0A12D72F0A16902B0A12DD2F0A16902B8A116D298A15902B8A11AA2996
:203660008A15902B8A11C4298A15902B0A12F32F0A16902B8A11DF298A15902B8A11F8293C
:203680008A15902B8A11192A8A15902B8A112B2A8A15902B8A115F2A8A15902B8A116D2A9E
:2036A0008A15902B8A11772A8A15902B8A11902A8A15902B8A119A2D8A15902B8A11E12D06
:2036C0008A15902B8A11042E8A15902B8A11432E8A15902B8A11742E8A15902B8A11A52EFE
:2036E0008A15902B8A11D22E8A15902B8A11E02E8A15902B0028902B8A11682F8A15902B09
:20370000EE28902B6F29902B8A11A92F8A15902B8A11CC2F8A15902B902B652AAC01AB0125
:203720008A150A16C52B840183131F30830583161F149F141F159F1107309C0033308312BA
:20374000E1001930E2000C30E3003330E4000A128A11882A0A168A150A128A11992B0A1634
:203760008A150A128A11782D0A168A150A12BA2B0A160A128A11AB2E0A168A150A122C2DAA
:203780000A168A1100288A15552AB12B6300FFFFFFFFFFFFFFFFFFFFFFFFFFFFFFFFFFFFFB
:2037A000FFFFFFFFFFFFFFFFFFFFFFFFFFFFFFFFFFFFFFFFFFFFFFFFFFFFFFFFFFFFFFFF29
:2037C000FFFFFFFFFFFFFFFFFFFFFFFFFFFFFFFFFFFFFFFFFFFFFFFFFFFFFFFFFFFFFFFF09
:2037E000FFFFFFFFFFFFFFFFFFFFFFFFFFFFFFFFFFFFFFFFFFFFFFFFFFFFFFFFFFFFFFFFE9
:203800000A108A100A15820746345234013446345434013455345034023444344E3402346D
:203820004C344B3401344D34443402344634573400344734543400344E3442340334503402
:203840004134013452344134013452345434013458345434013452344434003452345534C1
:2038600000345234433400344B345334053450344334053441344E340134543458340034FC
:203880005234583400344B34593406345334573404345334513405344B345934073444344E
:2038A000533400340A108A100A1582074134493431343B344134493432343B344B3432347F
:2038C00032343B344B3453343B34493446343B344B3459343B34463457343034303430348C
:2038E000303447345434303430344D34443433343B34423447343B34443453343B344D347B
:2039000044343B344C34533442345534533442344334573443345234523454344B343234CB
:2039200030343B340A108A100A1582071E341B341934173415341434133412341134103478
:203940000F340E340E340D340D340C340C340B340B340A340A340A34093409340934093472
:2039600008340834083408340834073407340734073407340734063406340634FFFFFFFF0F
:20398000FFFFFFFFFFFFFFFFFFFFFFFFFFFFFFFFFFFFFFFFFFFFFFFFFFFFFFFFFFFFFFFF47
:2039A000FFFFFFFFFFFFFFFFFFFFFFFFFFFFFFFFFFFFFFFFFFFFFFFFFFFFFFFFFFFFFFFF27
:2039C000FFFFFFFFFFFFFFFFFFFFFFFFFFFFFFFFFFFFFFFFFFFFFFFFFFFFFFFFFFFFFFFF07
:2039E000FFFFFFFFFFFFFFFFFFFFFFFFFFFFFFFFFFFFFFFFFFFFFFFFFFFFFFFFFFFFFFFFE7
:203A00000A148A100A1582074F34463446342034203441344334433431342134413443341E
:203A20004334323422344134433443343334233441344334433434342434413443344334AC
:203A400035342534413443344334363426344134433443343734273410340834003410345C
:203A60000934003410340A34003410340B3400340534323415340134053405340034413430
:203A80004E3400344134543400344134463400344934463400344E34423400344E345434BB
:203AA0000034503452340034523449345434003458344934543400344F3446340034533458
:203AC000503400345234583400340034003400340A148A100A15820700340034013400341B
:203AE00002340034083400340034013400340234003404340034083400341034003420343D
:203B0000043400340034403400344034003480341034003400340034003400340034403411
:203B2000003480340034C0341034003410344034103480341034C034003420344034603485
:203B40008034A034C034E0340034203440348034FF34FF34FF34FF340A148A100A158207F9
:203B60001F34043433340C34403409345A340734733405348D340334A6340234FF34013449
:203B80000A148A100A158207193401342A3402343A340334493404345B3405346D340634B2
:203BA0007F34073491340834A0340934B2340C34C4340D34FF340E34FF34FF34FF34FF3465
:203BC000FF34FF34FF34FF34FFFFFFFFFFFFFFFFFFFFFFFFFFFFFFFFFFFFFFFFFFFFFFFF31
:203BE000FFFFFFFFFFFFFFFFFFFFFFFFFFFFFFFFFFFFFFFFFFFFFFFFFFFFFFFFFFFFFFFFE5
:203C0000011A00110218000F0317000F0419000F05140000051F490106140000061F4901EA
:203C200007140000071F490108140000081F4901091F00040A1B00010B1B00020C132201B0
:203C40000C1F46010D1F00030E1321010E1F45010F1F00170F1F011A101F0018101F021AED
:203C60001106000112130C00121F450113135101131F450114135001141F45011517010274
:203C8000151F440116170101161F5501171F0023181F0024190DFD00191F53011A0D030064
:203CA0001A1F53011B1A000B1B1F54011C1A01111C1F00221E1F001C1F1F001D691F530173
:203CC000691F000F6F1F50016F1F0016431F0009431F0003431F4D016B1F0111671F4701E0
:203CE000671F000E5D1F13005D1F001F701F1600701F0014661F4101661F0021651F460186
:203D0000651F000C6A1F4C016A1F00106C1F1F006C1F00126D1F22006D1F00136E1F25005E
:203D20006E1F0015711F5201711F0017731F5801731F0018621F5201621F0009751F33009D
:203D4000751F000B631F5401631F000AA91F5301A91F000FAF1F5001AF1F0016831F0009C0
:203D6000831F0003831F4D01AB1F0111A71F4701A71F000E9D1F13009D1F001FB01F160061
:203D8000B01F0014A61F4101A61F0021A51F4601A51F000CAA1F4C01AA1F0010AC1F1F009F
:203DA000AC1F0012AD1F2200AD1F0013AE1F2500AE1F0015B11F5201B11F0017B31F580150
:203DC000B31F0018B41F3000B41F001AA21F5201A21F0009B51F3300B51F000BA31F54012E
:203DE000A31F000AA01F4101A01F0006A11F4201A11F0008BB1F3600BB1F0020E91F530100
:203E0000E91F000FEF1F5001EF1F0016C31F0009C31F0003C31F4D01EB1F0011E71F47019F
:203E2000E71F000EDD1F1300DD1F001FF01F1600F01F0014E61F1900E61F0021E51F1C0098
:203E4000E51F000CEA1F4C01EA1F0010EC1F1F00EC1F0012ED1F2200ED1F0013EE1F25001D
:203E6000EE1F0015F11F2800F11F0017F31F2C00F31F0018F41F3000F41F001AE21F520195
:203E8000FFFFFFFFFFFFFFFFFFFFFFFFFFFFFFFFFFFFFFFFFFFFFFFFFFFFFFFFFFFFFFFF42
:203EA000FFFFFFFFFFFFFFFFFFFFFFFFFFFFFFFFFFFFFFFFFFFFFFFFFFFFFFFFFFFFFFFF22
:203EC000FFFFFFFFFFFFFFFFFFFFFFFFFFFFFFFFFFFFFFFFFFFFFFFFFFFFFFFFFFFFFFFF02
:203EE000FFFFFFFFFFFFFFFFFFFFFFFFFFFFFFFFFFFFFFFFFFFFFFFFFFFFFFFFFFFFFFFFE2
:203F0000FFFFFFFFFFFFFFFFFFFFFFFFFFFFFFFFFFFFFFFFFFFFFFFFFFFFFFFFFFFFFFFFC1
:203F2000FFFFFFFFFFFFFFFFFFFFFFFFFFFFFFFFFFFFFFFFFFFFFFFFFFFFFFFFFFFFFFFFA1
:203F4000FFFFFFFFFFFFFFFFFFFFFFFFFFFFFFFFFFFFFFFFFFFFFFFFFFFFFFFFFFFFFFFF81
:203F6000FFFFFFFFFFFFFFFFFFFFFFFFFFFFFFFFFFFFFFFFFFFFFFFFFFFFFFFFFFFFFFFF61
:203F8000FFFFFFFFFFFFFFFFFFFFFFFFFFFFFFFFFFFFFFFFFFFFFFFFFFFFFFFFFFFFFFFF41
:203FA000FFFFFFFFFFFFFFFFFFFFFFFFFFFFFFFFFFFFFFFFFFFFFFFFFFFFFFFFFFFFFFFF21
:00000001FF
